:060000000A128A11FC2F18
:100F200083160313061486140615861506168616F0
:100F300006178617871307138712071283120313E6
:100F400087130713871207120610861006118611E1
:100F50000612861206138613061CAF2FB02FB52F6C
:100F60008713071787160716AC2F861CB82FB92FC3
:100F7000BE2F8717071387160716AC2F061DC12F24
:100F8000C22FC72F8713071387160716AC2F861D8E
:100F9000CA2FCB2FD02F8717071787120716AC2F12
:100FA000061ED32FD42FD92F8713071787120716A2
:100FB000AC2F861EDC2FDD2FE22F87170713871239
:100FC0000716AC2F061FE52FE62FEB2F871307130D
:100FD00087120716AC2F861FEE2FEF2FF42F8717DF
:100FE000071787160712AC2F8713071387120712EC
:100FF000AC2F0A128A11002883010A128A11902F3D
:02400E00BA3FB7
:00000001FF
